:020000040000FA
:0600000028EF01F01200E0
:020006000000F8
:08000800D9CFE6FFE1CFD9FFDB
:10001000030EE126050EF36E010EF3CFDBFF020E99
:10002000DB6A926A9468956A806A836A190EE66E42
:10003000E66A3C0EE66EB4EC00F0E552E552E5529D
:10004000010EE66E18EC01F0E552F9EC00F0DF6EFF
:10005000DF50300A28E0080A24E00F0A1FE0010AF6
:100060001AE0030A15E0010A10E0070A0BE0010A92
:1000700006E0030A01E019D0010E836E16D0030ECC
:10008000836E13D0070E836E10D00F0E836E0DD0CB
:100090001F0E836E0AD03F0E836E07D07F0E836ED5
:1000A00004D0836802D0836A00D0CAD74F0EAB1643
:1000B000AC9ACF0E9D16030EE15C02E2E16AE552B6
:0A00C000E16EE552E7CFD9FF120010
:0600CA00060EF66E000EAA
:1000D000F76E000EF86E00010900F550856F0900FB
:1000E000F550866F03E1856701D03DD00900F550DA
:1000F000806F0900F550816F0900F550826F09008B
:100100000900F550E96E0900F550EA6E0900090092
:100110000900F550836F0900F550846F090009004C
:10012000F6CF87F0F7CF88F0F8CF89F080C0F6FFE0
:1001300081C0F7FF82C0F8FF0001835302E18453BE
:1001400007E00900F550EE6E8307F8E28407F9D75F
:1001500087C0F6FF88C0F7FF89C0F8FF0001850758
:08016000000E865BBFD7120000
:08016800D9CFE6FFDACFE6FF74
:10017000E1CFD9FFE2CFDAFFAC6AAB6AFD0EDBB0AC
:10018000AC88DBA202D0AC8CAB8CDBB4AC8EDBA633
:1001900002D0AB8801D0AB8ADBB8AC849E98DBBAC6
:1001A000AB86DBAC02D09D8A01D09D9A9E9ADBAED5
:1001B00002D09D8801D09D98FB0EDB50AF6EFB0EE8
:1001C000FC0EDBCF03F003C002F0036A0250B06EF6
:1001D000AC8AAB8E949C948EAC50100B04E0AC5067
:1001E000800B01E1948CE552E5CFDAFFE7CFD9FF30
:0201F0001200FB
:0E01F200D9CFE6FFDACFE6FFE1CFD9FFE2CFAB
:10020000DAFFE652F20E00018A17ABAC03D08A91F6
:10021000ABB08A81ABB48A85ABB28A87AE50DF6E51
:10022000DF50E552E552E5CFDAFFE7CFD9FF120004
:10023000FF0EE350046E480E01D04C0EE76EE72E21
:10024000FED7E76AE72EFED7042EF7D7000012008C
:1002500015EE00F025EE00F0F86A019C65EC00F068
:0C0260003DEC01F004EC00F0FBD71200B4
:04026C0000EE00F0B0
:0A0270000F0EEE6AEA62FDD71200DD
:02027A00120070
:00000001FF
